:100000000C945C000C946E000C946E000C946E00CA
:100010000C946E000C946E000C946E000C946E00A8
:100020000C946E000C946E000C946E000C946E0098
:100030000C946E000C946E000C946E000C946E0088
:100040000C9488000C946E000C946E000C946E005E
:100050000C946E000C946E000C946E000C946E0068
:100060000C946E000C946E00000000080002010069
:100070000003040700000000000000000102040863
:100080001020408001020408102001020408102002
:10009000040404040404040402020202020203032E
:1000A0000303030300000000250028002B000000CC
:1000B0000000240027002A0011241FBECFEFD8E043
:1000C000DEBFCDBF21E0A0E0B1E001C01D92A930AC
:1000D000B207E1F70E94F1010C9401020C940000B8
:1000E00061E08DE00C94810161E08DE00E94BA0135
:1000F00068EE73E080E090E00E94F50060E08DE043
:100100000E94BA0168EE73E080E090E00C94F50084
:100110001F920F920FB60F9211242F933F938F933C
:100120009F93AF93BF938091010190910201A091A1
:100130000301B09104013091000123E0230F2D371A
:1001400020F40196A11DB11D05C026E8230F0296DB
:10015000A11DB11D20930001809301019093020124
:10016000A0930301B09304018091050190910601D1
:10017000A0910701B09108010196A11DB11D8093C6
:10018000050190930601A0930701B0930801BF9168
:10019000AF919F918F913F912F910F900FBE0F9034
:1001A0001F9018953FB7F894809105019091060132
:1001B000A0910701B091080126B5A89B05C02F3F6B
:1001C00019F00196A11DB11D3FBF6627782F892F19
:1001D0009A2F620F711D811D911D42E0660F771FDE
:1001E000881F991F4A95D1F70895CF92DF92EF9219
:1001F000FF92CF93DF936B017C010E94D200EB0151
:10020000C114D104E104F10489F00E9400020E94AB
:10021000D2006C1B7D0B683E734090F381E0C81ADE
:10022000D108E108F108C851DC4FEACFDF91CF9146
:10023000FF90EF90DF90CF900895789484B582601E
:1002400084BD84B5816084BD85B5826085BD85B57A
:10025000816085BDEEE6F0E0808181608083E1E829
:10026000F0E0108280818260808380818160808361
:10027000E0E8F0E0808181608083E1EBF0E0808164
:1002800084608083E0EBF0E0808181608083EAE736
:10029000F0E08081846080838081826080838081BF
:1002A000816080838081806880831092C10008957E
:1002B000833081F028F4813099F08230A1F00895E4
:1002C0008730A9F08830B9F08430D1F48091800073
:1002D0008F7D03C0809180008F7780938000089588
:1002E00084B58F7702C084B58F7D84BD08958091D9
:1002F000B0008F7703C08091B0008F7D8093B000F5
:100300000895CF93DF9390E0FC01E458FF4F2491D0
:10031000FC01E057FF4F8491882349F190E0880F5A
:10032000991FFC01E255FF4FA591B4918C559F4F49
:10033000FC01C591D4919FB7611108C0F8948C91CC
:10034000209582238C93888182230AC0623051F4E5
:10035000F8948C91322F309583238C938881822B53
:10036000888304C0F8948C91822B8C939FBFDF917B
:10037000CF9108950F931F93CF93DF931F92CDB723
:10038000DEB7282F30E0F901E859FF4F8491F901D9
:10039000E458FF4F1491F901E057FF4F04910023F7
:1003A000C9F0882321F069830E9458016981E02FF8
:1003B000F0E0EE0FFF1FEC55FF4FA591B4919FB7F2
:1003C000F8948C91611103C01095812301C0812B99
:1003D0008C939FBF0F90DF91CF911F910F91089544
:1003E00008950E941D010E94F0010E947000C0E06B
:1003F000D0E00E9474002097E1F30E940000F9CF42
:060400000895F894FFCFFF
:00000001FF
